:020000040000FA
:040000000000B8281C
:08000800A000030E8312A10009
:100010000A08A2008A010408A3000B1C1F28050877
:100020000B10851D1F28481F1A280730B00001300B
:10003000B100B200C81F1F28BB01BC01BD018C1C50
:10004000A5288C10B6184028BB1B33284208BD07D2
:100050000318BC0A0319BB0A4108BC070318BB0AF2
:100060004008BB0752284508BD070318BC0A0319FE
:10007000BB0A4408BC070318BB0A4308BB07522845
:10008000B61C52282814BA1F28103A1AA809B71A01
:10009000A809B719A809031428180310B70DB80D3B
:1000A000B90DBA0D361C6228B00A30080739031D95
:1000B000A528B2030319B103031DA5283308B10015
:1000C0003408B20035088207862988298A299029B0
:1000D0009629A229A729B829CA01CB0103104618DD
:1000E000CA07CA0CCB0CC618CA07CA0CCB0C4619D7
:1000F000CA07CA0CCB0CC619CA07CA0CCB0C461AC5
:10010000CA07CA0CCB0CC61ACA07CA0CCB0C461BB2
:10011000CA07CA0CCB0CC61BCA07CA0CCB0C4609B3
:10012000CC00CD010310CC0CCD0C4D08CB0703182F
:10013000CA0A4C08CA074B0D9516031C95124B0DA5
:100140001516031C15124A08930023088400220880
:100150008A00210E8300A00E200E09000630A400A4
:10016000A40BB0289F149F18B3281E08AF000800E6
:1001700087010730990091010430920093018316A2
:1001800002308C00F730910020309F00FF30920049
:100190000F3087003F308500083096008312003012
:1001A0008C00C8308B000C309500FF30C6008030CA
:1001B000C700B5010130B200B100B301B401B00114
:1001C000B601C801C809C901B701B801B901BA012E
:1001D000BA0ABD01BC01BB01BE013830BF00C0017D
:1001E000C101C201C301C401C501AE01AE0A0030A4
:1001F0008A002E080739FF3E03188A0A8200072961
:100200000F29252937293C294B29F628F6280130C2
:100210009F00AE20CA23BE00D124BF00552905305F
:100220009F00AE20043EE039A4002F08E0392406E8
:10023000031DF6280310AF0E0E30AF052F0CB500CE
:10024000073AB6100319B614F62809309F00AE20FD
:10025000D825B300DF26B4002F0836183329F83923
:10026000031D3614F628FC3903193610F628113010
:100270009F00AE20C600F62815309F00AE20FC3946
:10028000031D442904304929FF3AFC39031903307E
:10029000FF3AC700552919309F00AE20C800F62844
:1002A0001D309F00AE20C900F628AC0103103E0CA3
:1002B000AA003F0CAB00AC0C4708D2006F214E08DF
:1002C000C0004F08C1005008C2004709D2006F218A
:1002D0004E08C3004F08C4005008C500F628D101DD
:1002E0001830AD002A08CE002B08CF002C08D00013
:1002F000500DCF0DCE0DD10DD00D5208D1020318E7
:100300005014501CD107AD0B782908003B086C280D
:100310003B096C28BB1B8E2900306C28FF306C28F1
:1003200003103C0D3B0DBB1BFF3A6C2803103C0D2A
:100330003B0DBA21A5000310A50CA5172508BB1B72
:10034000FF3A6C283B08BA21FF3AA5006C283B1BFA
:10035000B6293C08A5003B08A6000310A50DA60D74
:10036000A50D260DC222BB1BFF3A6C2880306C28DD
:100370003A086C28A50001308A002508C23E0318FF
:100380008A0A820000340334063409340D341034F0
:100390001334163419341C341F34223425342934D0
:1003A0002C342F343234353438343B343E344134F9
:1003B000443447344A344D34503453345634593429
:1003C0005C345F346234643467346A346D3470345E
:1003D0007334753478347B347E348034833486349B
:1003E00088348B348E3490349334953498349A34E2
:1003F0009D349F34A234A434A734A934AB34AE3432
:10040000B034B234B434B734B934BB34BD34BF348F
:10041000C134C334C534C734C934CB34CD34CF34FC
:10042000D134D234D434D634D734D934DB34DC3478
:10043000DE34DF34E134E234E434E534E734E83404
:10044000E934EA34EC34ED34EE34EF34F034F134A2
:10045000F234F334F434F534F634F734F734F83452
:10046000F934F934FA34FB34FB34FC34FC34FD3415
:10047000FD34FD34FE34FE34FE34FF34FF34FF34EB
:10048000FF34FF34FF34FF34FF34FF34FF34FF34D4
:10049000FE34FE34FE34FD34FD34FD34FC34FC34D3
:1004A000FB34FB34FA34F934F934F834F734F734E4
:1004B000F634F534F434F334F234F134F034EF3408
:1004C000EE34ED34EC34EA34E934E834E634E5343F
:1004D000E434E234E134DF34DE34DC34DB34D93488
:1004E000D734D634D434D234D034CF34CD34CB34E2
:1004F000C934C734C534C334C134BF34BD34BB344C
:10050000B934B634B434B234B034AD34AB34A934C5
:10051000A634A434A2349F349D349A34983495344C
:10052000933490348E348B348834863483348034DE
:100530007E347B3478347534733470346D346A347B
:100540006734643462345F345C3459345634533421
:1005500050344D344A344734443441343E343B34CF
:100560003834353432342F342B3428342534223483
:100570001F341C3419341634133410340C34093439
:1005800006340334A50002308A002508CA3E031849
:100590008A0A820081348134813481348134813407
:1005A00081348134813481348134813481348134A3
:1005B000813481348134823482348234823482348E
:1005C0008234823482348234823483348334833478
:1005D000833483348334843484348434843484345E
:1005E0008434853485348534853486348634863441
:1005F0008634873487348734873488348834893420
:1006000089348A348A348B348B348C348C348D34F2
:100610008D348E348E348F348F34903490349134C2
:10062000913492349334943494349534963497348A
:10063000983499349A349B349C349D349E349F343E
:10064000A034A234A334A534A634A834A934AB34DE
:10065000AC34AE34AF34B134B234B434B634B8346C
:10066000BA34BC34BE34C034C234C534C734CA34DE
:10067000CC34CF34D134D434D734DA34DD34E0342C
:10068000E334E734EA34EE34F134F534F834FB344F
:10069000FD34FF34FD34FB34F834F534F134EE34FA
:1006A000EA34E734E334E034DD34DA34D734D434B4
:1006B000D134CF34CC34CA34C734C534C234C03456
:1006C000BE34BC34BA34B834B634B434B234B134D1
:1006D000AF34AE34AC34AB34A934A834A634A5342A
:1006E000A334A234A0349F349E349D349C349B3474
:1006F0009A349934983497349634953494349434A5
:100700009334923491349134903490348F348F34C4
:100710008E348E348D348D348C348C348B348B34D5
:100720008A348A34893489348834883487348734E5
:1007300087348734863486348634863485348534E9
:1007400085348534843484348434843484348434E7
:1007500083348334833483348334833482348234E3
:1007600082348234823482348234823482348234D9
:1007700081348134813481348134813481348134D1
:1007800081348134813481348134813481348134C1
:100790008134813403308A002F08D13E03188A0A3D
:1007A000820000340034003400340034003400345B
:1007B0000034003400340034003400340034003499
:1007C0000034003400340034003400340034003489
:1007D0000034003400340034003400340034003479
:1007E0000034003400340034003400340034003469
:1007F0000034003400340034003400340034003459
:100800000034003400340034003400340034003448
:100810000034003400340034003400340034003438
:100820000034003400340034003400340034003428
:100830000034003400340034003400340034003418
:100840000034003400340034013401340134013404
:1008500001340134013401340134013401340134F0
:1008600001340134013401340134013401340134E0
:1008700001340134013401340134013401340134D0
:1008800001340134013401340234023402340234BC
:1008900002340234023402340234023402340234A8
:1008A0000234023402340234023402340234033497
:1008B0000334033403340334033403340334033480
:1008C000033403340334033404340434043404346C
:1008D0000434043404340434043404340534053456
:1008E000053405340534053405340534053406343F
:1008F0000634063406340634063406340734073426
:10090000073407340734073408340834083408340B
:100910000834093409340934093409340A340A34EE
:100920000A340A340A340B340B340B340B340C34D1
:100930000C340C340D340D340D340D340E340E34AF
:100940000E340F340F340F3410341034103411348B
:100950001134123412341234133413341434143462
:100960001534153415341634163417341734183436
:10097000193419341A341A341B341B341C341D3402
:100980001D341E341F341F342034213421342234CA
:100990002334243424342534263427342834293489
:1009A0002A3404308A002F08D83E03188A0A8200AD
:1009B0002B342C342D342E342F3430343134323423
:1009C0003334343435343734383439343A343C34CD
:1009D0003D343E3440344134423444344534473469
:1009E00048344A344C344D344F34513452345434F6
:1009F000563458345A345C345E346034623464346F
:100A0000663469346B346D347034723475347734D1
:100A10007A347C347F348234853488348B348E3419
:100A20009134943497349A349E34A134A534A83444
:100A3000AC34B034B434B834BC34C034C434C83446
:100A4000CD34D134D634DA34DF34E434E934EE341E
:100A5000F334F934FE34043409340F3415341B34C0
:100A6000213428342E3435343C3442344A34513421
:100A70005834603467346F34773480348834903439
:100A80009934A234AB34B534BE34C834D234DC34F7
:100A9000E734F134FC34073413341E342A3436344A
:100AA00043344F345C346A34773485349334A2341D
:100AB000B034BF34CF34DF34EF34FF34103421345A
:100AC00033344434573469347D349034A434B934E5
:100AD000CD34E334F8340F3425343D3454346D349C
:100AE00086349F34B934D334EE340A342634433454
:100AF00061347F349E34BD34DD34FE3420344234DE
:100B000065348934AE34D334F93420344834713404
:100B10009B34C534F1341E344B347934A934DA347F
:100B20000B343E347234A734DD3414344C34863400
:100B3000C134FD343B347A34BA34FC343F34843429
:100B4000CA3412345B34A634F23441349134E23482
:100B500036348B34E2343B349634F3345234B33489
:100B600016347C34E3344D34B934283499340C349D
:100B70008234FB347634F4347534F8347F340834FA
:100B800094342434B6344C34E53481342134C434C0
:100B90006B341634C43476342C34E634A4346634DE
:100BA0002D34F734C7349A34733450343234193412
:100BB00005308A002F08DF3E03188A0A820030348D
:100BC0002F342E342D342C342B342A342934293428
:100BD000283427342634253424342434233422344E
:100BE0002134213420341F341F341E341D341D346D
:100BF0001C341C341B341A341A3419341934183484
:100C00001834173417341634163415341534153493
:100C1000143414341334133412341234123411349F
:100C2000113411341034103410340F340F340F34A5
:100C30000E340E340E340D340D340D340D340C34AA
:100C40000C340C340C340B340B340B340B340B34A9
:100C50000A340A340A340A340934093409340934A8
:100C600009340934083408340834083408340834A2
:100C7000073407340734073407340734073406349D
:100C80000634063406340634063406340634063494
:100C9000053405340534053405340534053405348C
:100CA0000534053404340434043404340434043482
:100CB0000434043404340434043404340434033475
:100CC000033403340334033403340334033403346C
:100CD000033403340334033403340334033403345C
:100CE0000334033402340234023402340234023452
:100CF0000234023402340234023402340234023444
:100D00000234023402340234023402340234023433
:100D10000234023402340234023402340234023423
:100D20000234023401340134013401340134013419
:100D3000013401340134013401340134013401340B
:100D400001340134013401340134013401340134FB
:100D500001340134013401340134013401340134EB
:100D600001340134013401340134013401340134DB
:100D700001340134013401340134013401340134CB
:100D800001340134013401340134013401340134BB
:100D900001340134013401340134013401340134AB
:100DA000013401340134013401340134013401349B
:100DB000013401340134013401340134013406308A
:100DC0008A002F08E63E03188A0A82009C34973472
:100DD00097349D34A834B934CF34E93409342D34F0
:100DE00056348434B634ED3428346734AA34F234BB
:100DF0003D348C34DF3436349034EE344F34B434F4
:100E00001C348734F6346734DC345434CE344C34F8
:100E1000CC344F34D4345D34E834753405349734ED
:100E20002B34C2345B34F73494343434D5347934CD
:100E30001F34C63470341B34C83477342834DA3461
:100E40008E344434FB34B4346E342A34E734A6345C
:100E500066342834EA34AF3474343B340334CC344D
:100E6000963461342E34FC34CA349A346B343D34B5
:100E70001034E334B8348E3464343C341434ED34F8
:100E8000C734A2347E345A3437341534F434D3346E
:100E9000B3349434753458343A341E340234E6345E
:100EA000CB34B13497347E3465344D3436341F340A
:100EB0000834F234DC34C734B2349E348A347734A4
:100EC000643451343F342D341C340B34FA34EA3456
:100ED000DA34CA34BB34AC349D348F348134733447
:100EE000663459344C343F34333427341B34103493
:100EF0000434F934EE34E434D934CF34C534BC345A
:100F0000B234A934A03497348E3486347D347534A9
:100F10006D3465345E3456344F34483441343A3499
:100F200033342D34263420341A3414340E34083437
:100F30000234FD34F734F234ED34E834E334DE3493
:100F4000D934D534D034CC34C734C334BF34BB34B3
:100F5000B734B334AF34AB34A834A434A1349D34A3
:100F60009A349734933490348D348A34873484346B
:100F700081347F347C3479347734743472346F3410
:100F80006D346B34683466346434623460345E3497
:100F90005C345A34583456345434523451344F3407
:100FA0004D344C344A344834473445344434423464
:100FB000413440343E343D343C343A3439343834AE
:0C0FC000373436343434333432343134B6
:02400E00C230BE
:00000001FF
